:100000000C9480020C94EC230C949D020C949D02A1
:100010000C949D020C949D020C949D020C949D02E4
:100020000C949D020C949D020C9406290C94D929E1
:100030000C9452220C949D020C949D020C949D02EF
:100040000C949D020C949D020C949D020C949D02B4
:100050000C949D020C940A230C949D020C949D0216
:100060000C949D020C949D020C949D020C949D0294
:100070000C949D020C949D020C949D020C949D0284
:100080000C949D020C949D020C949D020C949D0274
:100090000C949D020C949D020C949D020C949D0264
:1000A0000C949D020C949D020C949D022900140056
:1000B0001A0008001500170000002B0004001600AD
:1000C000070009000A000000E1001D001B000600F7
:1000D000190005000000E000E200E30021522C417D
:1000E000000000001C0018000C00120013004C005F
:1000F0002A000B000D000E000F0034000000280045
:10010000110000001000360037003800E5002A42D8
:1001100000000000E700E6002252E40035001E0067
:100120001F002000210022000000007C2378257899
:100130002778A9002F0000002178247826782878D5
:10014000AA002F0200002078010001000100010038
:1001500000000000230024002500260027002D00B9
:100160002E00300021002200230033000000010097
:10017000300200001E001F002000520001004C0051
:10018000000000002700500051004F0035021E0201
:100190001F022002210222020000010001000100D2
:1001A00049004B004A0000000100010001004C0022
:1001B0004E004D00000001000100010001004C0054
:1001C00000000000230224022502260227022D023D
:1001D0002E020100010001000100330200000100B5
:1001E0000100000001000100010001000100010008
:1001F0000000000001000100010001001E0F0500C9
:10020000047F3F1F643214643214783C1E1E140AAB
:10021000052223252628292A2C2D2F303233353646
:10022000383A3B3D3E4042434547494A4C4E505187
:10023000535557595A5C5E6062646668696B6D6FAE
:1002400071737577797B7D7F81838587898A8C8EB1
:1002500090929496989A9C9E9FA1A3A5A7A8AAACB9
:10026000AEAFB1B3B4B6B8B9BBBCBEBFC1C2C3C5F3
:10027000C6C7C9CACBCCCDCED0D1D2D2D3D4D5D695
:10028000D7D7D8D9D9DADADBDBDBDCDCDCDCDCDDC8
:10029000DDDDDDDCDCDCDCDCDBDBDBDADAD9D9D8AC
:1002A000D7D7D6D5D4D3D2D2D1D0CECDCCCBCAC944
:1002B000C7C6C5C3C2C1BFBEBCBBB9B8B6B4B3B173
:1002C000AFAEACAAA8A7A5A3A19F9E9C9A9896940E
:1002D00092908E8C8A89878583817F7D7B797775E3
:1002E00073716F6D6B6968666462605E5C5A5957C2
:1002F000555351504E4C4A4947454342403E3D3B81
:100300003A3836353332302F2D2C2A29282625230A
:1003100022FFAA7F554000010101010101010101F5
:1003200002020202020202020203030303030303A6
:100330000304040404040404050505050506060673
:100340000606070707070708080808090909090A30
:100350000A0A0B0B0B0C0C0C0D0D0D0E0E0E0F0FD5
:100360000F10101111111212131314141515161663
:100370001717181819191A1A1B1B1C1D1D1E1E1FD2
:100380002020212222232424252626272829292A21
:100390002B2C2D2D2E2F3031323233343536373849
:1003A000393A3B3C3D3E3F40414243444546474845
:1003B000494A4C4D4E4F50515354555658595A5B1B
:1003C0005D5E5F616264656668696B6C6D6F7072BB
:1003D000737577787A7B7D7E8082838587888A8C27
:1003E0008E8F91939596989A9C9EA0A2A3A5A7A95B
:1003F000ABADAFB1B3B5B7BABCBEC0C2C4C6C9CB52
:10040000CDCFD1D4D6D8DBDDDFE2E4E7E9EBEEF007
:10041000F3F5F8FAFDFF100346006F007500720057
:1004200069006500720000000E034B006500650066
:10043000620069006F0000000403090409023B0028
:10044000020100A0FA0904000001030101000921D2
:10045000110100012244000705810308000109047D
:1004600001000103000000092111010001223200F6
:10047000070582032000011201000200000008109D
:10048000CB471200010102000105010980A101858D
:100490000319012AB700150126B7009501751081CF
:1004A00000C0050C0901A101850419012AA002154B
:1004B0000126A002950175108100C005010906A161
:1004C00001050719E029E715002501950875018147
:1004D000029501750881010507190029FF150026FD
:1004E000FF0095067508810005081901290515000A
:1004F0002501950575019102950175039101C000D3
:1005000011241FBECFEFDAE0DEBFCDBF11E0A0E0C7
:10051000B1E0E8E0FCE502C005900D92AE3EB10707
:10052000D9F723E0AEEEB1E001C01D92A937B207C2
:10053000E1F70E9482150C94942D0C9400008330F6
:10054000B8F46830A8F4473098F4E42FF0E097E06E
:10055000699FE00DF11D112498E3899FE00DF11DC5
:100560001124EE0FFF1FE455FF4F859194910895DC
:1005700081E090E008950E949F02089581E008952F
:100580000E94BE02089581E008950E94BE0208956F
:100590000E94C502089508950E94CB020895A6E026
:1005A000B0E0E5EDF2E00C94402C49835A839E8341
:1005B0003091F50189819A8131111AC03E8133232E
:1005C00099F0222389F00E94DD08182F682F898175
:1005D0009A810E94B90869817A81812F0E94A80FAF
:1005E0002696E3E00C945C2C0E94CB08182FF3CFE6
:1005F0000E94DD0869817A81F1CFFC01262F4081BC
:10060000518162817381848195810E94CF02089516
:10061000CF93DF93D82FC92F61E00E94FD026D2F89
:100620007C2F0E94C002DF91CF910895CF93DF937A
:10063000D82FC92F60E00E94FD026D2F7C2F0E94F1
:10064000CC02DF91CF91089581E008950E942403A8
:100650000895CF93C82F0E948B078C2F0E942603EA
:100660002FEF84E39CE0215080409040E1F700C0F0
:100670000000CF91089581E00E9429030E942E235B
:10068000089580E00E9429030E943F2308950F935C
:100690001F93CF93DF938C0161E00E94FD02EC0178
:1006A000F801858181110E94F41DB801CE010E94DC
:1006B000C8028823E1F1B801CE010E94F12088230D
:1006C000B1F1B801CE010E94A61F882381F1B801C3
:1006D000CE010E947B1F882351F1B801CE010E94F8
:1006E000141E882321F1F8018581882381F0CA3501
:1006F000FCE7DF0739F178F4C130ECE7DE07F9F009
:10070000C330FCE7DF07C9F0C115DC4771F0C80151
:100710000E94C3020DC0CB35ECE7DE07B1F0CC354B
:10072000DC47A9F70E94DF0CF2CF0E943B0380E078
:10073000DF91CF911F910F9108950E94F10C0E94BB
:100740004103F5CF0E94E90CE2CF0E94ED0CDFCF10
:100750000E942F220E94CF0308950E94D3030E947B
:1007600034220895089581E008950895CF93DF938A
:10077000D82F0E94B303C82F882319F08D2F0E9411
:10078000B5038C2FDF91CF9108950895CF93C82F93
:100790000E94B2038C2F0E94B603CF91089580E08F
:1007A0000E94C60308950E9437210E94C60308953F
:1007B000CF930E943721C82F8091F0018C1779F0D8
:1007C000C093F0010E94BE226093F1017093F20188
:1007D0008093F3019093F4018C2F0E94C603CF9174
:1007E0000895ADE0B0E0E7EFF3E00C94412C4887CA
:1007F00059876A877B878C879D8791110E941C0C83
:100800001F8286E0FE013896DE01119601900D925E
:100810008A95E1F78D8181110DC029813A814B8143
:100820005C816D817E818F810E94620B2D96E2E05A
:100830000C945D2CCE0101960E9408038111EDCF2E
:10084000F5CFFC018481813021F4808191810E9467
:100850000F090895CF93C82F8823C9F08238C9F4AF
:100860000E944B2181FD13C089E30E94F6210E9462
:100870008D0C2FEF37EE83E0215030408040E1F7C0
:1008800000C0000089E30E94FE210E948D0CCF91E0
:1008900008958338A1F40E944B2180FDF8CF83E5B1
:1008A0000E94F6210E948D0C9FEF21EE34E09150C2
:1008B00020403040E1F700C0000083E5E4CF8438F9
:1008C000A1F40E944B2182FDE2CF87E40E94F62131
:1008D0000E948D0C8FEF91EE24E0815090402040DB
:1008E000E1F700C0000087E4CECF8CEF8C0F813A97
:1008F00098F48C2F0E942A1F8111C9CF8C2F0E943F
:10090000B921882329F08C2F0E94FE210E948D0C92
:100910008C2F0E94F621B9CF80E28C0F883048F4EA
:10092000C77081E001C0880FCA95EAF70E94FD0BED
:10093000ACCF8BE58C0F833038F42C2F2452330B43
:10094000C9010E945921A3CFC85ACB3108F09FCFCB
:10095000EC2FF0E0EE0FFF1FEB5BFE4F80819181EB
:100960000E947F2194CF882309F44DC0823879F406
:100970000E944B2181FF47C089E30E94F6210E941B
:100980008D0C89E30E94FE210E948D0C089583380E
:1009900059F40E944B2180FF36C083E50E94F62166
:1009A0000E948D0C83E5EECF843859F40E944B21D0
:1009B00082FF29C087E40E94F6210E948D0C87E403
:1009C000E1CF9CEF980F913AE8F290E2980F9830BF
:1009D00050F4877091E001C0990F8A95EAF7892F4A
:1009E0000E94030CD1CF9BE5980F933028F480E050
:1009F00090E00E9459210895885A8B3120F480E0BC
:100A000090E00E947F2108951F93CF93DF93182FCA
:100A1000EB010E942A04209739F4812F0E94B3042D
:100A2000DF91CF911F9108958FE99FE00197F1F732
:100A300000C000002197EFCF60E070E0893311F42F
:100A400060E570E00E9404050895882321F00E946B
:100A5000FD0B0E948D0C0895882321F00E94030C49
:100A60000E948D0C0895A0E0B0E0E9E3F5E00C945D
:100A70003B2C6C01D62FC72FFC010581F680F29428
:100A80008FE0F8220E94F20BE82E8823F9F0E02E86
:100A90000023E1F08C2F807F803461F080E28D0FA5
:100AA0008830A0F18C2F807E803221F4D23070F11A
:100AB000FF2061F180911F0382FF28C082E00E9425
:100AC000B20C0E94F20B91E0E82EE9268C2F829561
:100AD0008F70883009F4E7C0B0F58430C8F41C2F5B
:100AE0001F70823008F440C0C07FC03211F01295F0
:100AF000107FDD2309F467C0D13009F497C00023CB
:100B000009F4A3C0FF2009F47AC041C0E12CDECF74
:100B1000843009F4ABC0EE2089F00E94EE0B80FD1A
:100B20000DC0F60115820E94E80B0E941608C6014E
:100B30000E9456070E94E80B0E942608CDB7DEB738
:100B4000E8E00C94572C893009F424C18A5F8F7037
:100B5000823008F7D23F09F02EC18C2F8F7101111E
:100B600027C10E941608CEC0C03110F01295107F28
:100B7000002399F0112359F080E28D0F883010F096
:100B8000D11107C0812F0E94FD0B0E948D0C8D2F6B
:100B900028C0812F0E940E0CF8CF8D2F0E94B30425
:100BA000112309F4B8CF80E28D0F883010F0D111F5
:100BB00004C0812F0E94030C03C0812F0E94140CDB
:100BC0000E948D0CA8CF80911F0382FD14C00023CA
:100BD00059F0112329F0812F0E94FD0B0E948D0CEA
:100BE00080E00E942A0497CF80E00E94B304112382
:100BF00009F491CFDECF002369F0F11004C0812FFA
:100C00000E94250588CFF1E0FF1285CF812F0E9439
:100C1000340C81CFF1107FCF812F0E942C05812FC2
:100C20000E94400C812F0E94230C75CF002329F0D5
:100C300025E02F1508F46FCFE2CF84E08F1508F47C
:100C40006ACF812F0E942C0566CFFF20D1F3D933C4
:100C500049F49FEFE7EEF3E09150E040F040E1F718
:100C600000C000008D2F0E94B30455CF8C2F8695B5
:100C700086958370882369F0813009F04CCF8D2FE1
:100C80009C2F9370011102C080E090E00E947F21B0
:100C900042CF8D2F9C2F9370011102C080E090E015
:100CA0000E94592138CF8C2F8370811139C00111D6
:100CB00029C04D2F429546954770440F440F2D2F64
:100CC0002F7030E0042E02C0220F331F0A94E2F787
:100CD00080E090E0D4FF09C08FE090E002C0880F70
:100CE000991F4A95E2F780959095C695C695C37071
:100CF000822B932BC23071F0C33079F0C13039F0C0
:100D00000E94E6070E9437210E94C60304CF0E947A
:100D1000DD07F8CF0E94EF07F5CF0E94DA07F2CF88
:100D2000002361F1C0FFEECF4D2F429546954770ED
:100D3000440F440F2D2F2F7030E0042E02C0220FDD
:100D4000331F0A94E2F780E090E0D4FF09C08FE0FF
:100D500090E002C0880F991F4A95E2F78095909520
:100D6000C695C695C370822B932BC23069F0C330F1
:100D700071F0C13031F00E945108C4CF823010F2BE
:100D8000D3CF0E944808BECF0E945A08BBCF0E9412
:100D9000FE07B8CFCF70002339F08C2F0E941608C1
:100DA0008D2F0E942505AECF8D2F0E942C058C2FF4
:100DB0000E942608A7CFD33F70F4D03FB9F0D13FAF
:100DC00089F1002309F449C0FF2009F443C08D2FA5
:100DD0000E942A0497CFD33FB9F0D43FF9F0011114
:100DE000F3CFF11047C08C2F8F71E2CF002349F071
:100DF00024E02F1508F486CF8C2F8F710E943808BD
:100E000081CF85E0F816F6CF002329F08C2F8F7163
:100E10000E940A0877CF0E94050874CF80911F03B3
:100E200082FD05C08C2F8F71002311F29ACE002312
:100E300031F063E08C2F8F710E94940C63CF81E0BE
:100E40000E94B20C91E09F1508F05CCF82E00E94F6
:100E5000B20C58CF8C2F8F7184CEFF2021F2D93362
:100E600049F4EFEFF7EE23E0E150F0402040E1F7E6
:100E700000C000008D2F0E94B30444CF0F931F9336
:100E8000CF93DF93EC01688179818D810E941C09E9
:100E90008C010E9463080E94D907B801CE010E940C
:100EA0003305DF91CF911F910F910895CF93DF9379
:100EB000EC018C81882399F0CE010E9447038111B7
:100EC00011C00E94F20B882351F08D81882339F0E4
:100ED00080911F0382FF03C082E00E94B20CDF9169
:100EE000CF910895CE010E943E07CE010E941603C5
:100EF000F6CF80E090E00E94592180E090E00E94CF
:100F00007F210E941C0C0E948D0C08950E940622D5
:100F10000E94790708950E940B0C0E94860708958D
:100F2000282F92959F70963091F060F4925F9F7099
:100F3000923030F481E0203F79F030F4283E30F0F8
:100F400080E008959A5FF3CF243FD1F7089581E0C0
:100F5000283EE0F3213FF9CF0895FC0184818823E6
:100F600039F0808191810E940F090E9490070895B5
:100F700080E00895A6E0B0E0E0ECF7E00C94412CAE
:100F80002696E2E00C945D2CA7E0B0E0EAECF7E0F6
:100F90000C94412C2796E2E00C945D2C08950E945D
:100FA000CE0708950E94CF079093150280931402F4
:100FB000089508950E94D207089520911402309157
:100FC0001502822B932B0E94D207089520911402C0
:100FD00030911502822393230E94D2070895209115
:100FE000140230911502822793270E94D207089598
:100FF0000E94CE0708950E94F80708950E94FB07FB
:101000009093130280931202089580E090E00E9472
:10101000FE07089521E030E0A90102C0440F551FEA
:101020008A95E2F7CA010E94FE07089521E030E0A8
:1010300002C0220F331F8A95E2F78091120290912D
:101040001302822B932B0E94FE07089521E030E0CB
:1010500002C0220F331F8A95E2F7209530958091C8
:10106000120290911302822393230E94FE07089597
:1010700021E030E002C0220F331F8A95E2F7809111
:10108000120290911302822793270E94FE0708956F
:101090002091120230911302822B932B0E94FE07A3
:1010A00008952091120230911302822393230E940B
:1010B000FE07089520911202309113028227932790
:1010C0000E94FE07089508959B01677091E001C09A
:1010D000990F6A95EAF763E0369527956A95E1F7E7
:1010E000220F331F220F331FFA01E20FF31F40E0DC
:1010F00050E0682F70E08191DF0111979B01042E71
:1011000002C0369527950A94E2F721702195282789
:10111000292328272C934F5F5F4F4430510559F7FF
:1011200008959C01982F977083E0369527958A95AE
:10113000E1F7220F331F220F331FFB01E20FF31FD2
:1011400040E050E080E0219130E0092E02C0369569
:1011500027950A94E2F721703327042E01C0220F4D
:101160000A94EAF7822B4F5F5F4F4430510559F7DD
:101170000895282F862F983068F4273058F4622F6E
:1011800070E027E0929F600D711D112446EF51E041
:101190000E9464080895292F983068F4873058F425
:1011A00090E066EF71E037E0239F800D911D1124E0
:1011B0000E949108089580E00895A0E0B0E0E3EE79
:1011C000F8E00C943A2C8C01E0901202F09013029B
:1011D0008091140290911502E82AF92ACFE0D0E01C
:1011E000CC24C394D12CC6010C2E02C0880F991FA9
:1011F0000A94E2F78E219F21892B49F4219798F7D1
:10120000B12C8B2DCDB7DEB7E9E00C94562CBC2E5B
:10121000B8018C2F0E94B40F019781F3F2CFCF93C6
:10122000DF93D82FC92F0E94DD086D2F7C2F0E94DD
:10123000B40FDF91CF9108951F93CF93DF93162FB3
:10124000D72F9091F501992341F0862F972F0E9477
:101250000F09DF91CF911F910895882381F0862F88
:10126000972F0E94DD08C82F682F812F9D2F0E9485
:10127000B908612F7D2F8C2F0E94B40FEACF862FE3
:10128000972F0E94CB08C82FF4CF0F931F93CF93B3
:10129000E0911602C7E0809117028E1304C0CF912F
:1012A0001F910F9108950E2F10E0CE9FF001112491
:1012B000E85EFD4F208131814281538164817581D7
:1012C00086810E94C407F8013196E770E4CF20912F
:1012D000500230915102409152025091530260915C
:1012E000540270915502809156020E94C4070895DD
:1012F00080915602803178F480915502882359F00C
:10130000E091160220911702309151024091500253
:1013100057E02E1301C008956E2F70E05E9FF0011C
:101320001124DF01A85EBD4F14968C911497882379
:1013300061F111968C911197831327C08C918413BE
:1013400024C015968C91159781111FC012968D910E
:101350009C91A0915202B09153028A1B9B0B883C36
:10136000910598F4809156028F70806180935602A7
:10137000E25EFD4F80818F708061808380E592E026
:101380000E9456070E9445090895FB013196E770B7
:10139000C0CFE09116029091170227E0E91302C036
:1013A00080E00895AE2FB0E02E9FF0011124E85E9A
:1013B000FD4F3181361306C03081381303C03581AB
:1013C000341304C0FD013196E770E8CF81E0089541
:1013D0008F929F92AF92BF92DF92EF92FF920F9304
:1013E0001F93CF93DF93CDB7DEB72D970FB6F89449
:1013F000DEBF0FBECDBF8C0186E0F801DE0118967E
:1014000001900D928A95E1F7F801E080F580A280C5
:10141000B380848190E5892E92E0992E90915402B8
:1014200091111BC0882309F4FCC0FF2009F43DC1C1
:10143000C8010E94AD07882309F437C187E0F8018D
:10144000D40101900D928A95E1F7C4010E94210414
:101450000E9478090E946709E4C0D090550220914B
:10146000520230915302A501421B530BDD2009F4B7
:10147000DBC0483C510508F0A6C0882309F4D1C060
:1014800090915102918080915602803108F06BC09A
:10149000991228C0909150029E1124C0F1105DC095
:1014A0008F708061809356020E94670980E592E008
:1014B0000E94560780915602F8018683F12C8F2DE9
:1014C0002D960FB6F894DEBF0FBECDBFDF91CF9142
:1014D0001F910F91FF90EF90DF90BF90AF909F9082
:1014E0008F900895F11039C040E0692D8E2D0E9433
:1014F000C90940E0692D8E2D0E94C909F82E81117D
:10150000DDCF888599850E940F09292F22952F709C
:10151000903450F49F70223080F0992399F0F801B4
:101520009681903178F4CBCF2A5F2F70223078F0FB
:10153000C8010E945607FD2CC2CF992319F08823B9
:1015400009F4BDCF805E883008F4B9CFF1CF803F79
:1015500008F4B5CF815F8230F7CF80915602816069
:1015600080935602ABCF991207C0909150029E1102
:1015700003C0FF2009F479C0C8010E94AD07882389
:1015800009F493C0FF2009F490C080915602803284
:1015900088F020915002309151023A832983BC8215
:1015A000AB82909154029D831E828F83CE0101965F
:1015B0000E94560787E0F801A0E5B2E001900D9285
:1015C0008A95E1F745CF909156029031A0F4488575
:1015D00059856A857B858C859D850E94BA0780E543
:1015E00092E00E94560787E0F40111928A95E9F78C
:1015F0000E94670963CF8823A1F020915102818165
:101600002813BACF809150028E11B6CFF110B4CF0B
:101610009683C8010E94560787E0F40111928A95CB
:10162000E9F7FF24F3944BCF483C510508F041C043
:101630008823B9F3FF20C9F1909151028181981359
:101640002AC0809150028E1126C08091560280FDE2
:1016500019C08031B8F08683807F803F39F0868161
:10166000982F907F905F8F70892B8683C8010E948E
:10167000560787E0F801A0E5B2E001900D928A9547
:10168000E1F7E8CE87E0F801A0E5B2E001900D9225
:101690008A95E1F7C6CFC8010E94AD0781118ACFB4
:1016A00080915602816080935602C8010E945607BD
:1016B000B8CF488559856A857B858C859D850E9434
:1016C000BA0791CFAEE0B0E0E8E6FBE00C94402C26
:1016D000288739874A875B876C877D878E87CE010D
:1016E00008960E94E8098823B1F06C85662341F0D2
:1016F000288539854A855B857D858E850E94C4074E
:1017000017E0809116029091170289133EC02E9621
:10171000E3E00C945C2C87E0FE013896DE01119624
:1017200001900D928A95E1F72091170240911602DF
:101730008C85882329F330E0C901019687709927A9
:1017400050E08417950799F097E0929FD001939FFE
:10175000B00D1124A85EBD4FFE01319601900D928F
:101760009A95E1F7809317020E944509C9CF0E941C
:101770008B07109217021092160287E0E0E5F2E064
:10178000DF011D928A95E9F7BBCF189FC001112494
:10179000885E9D4F0E94E809882309F4B8CFE09144
:1017A00016021E9FF0011124E85EFD4F2081318159
:1017B000428153816481758186810E94C407809132
:1017C000160290E00196877099278093160299CFB0
:1017D00080915F02869586958695089580915F0237
:1017E0008770089590915F02977081E0911101C018
:1017F00080E0089580916B02089590916B02982B80
:1018000090936B020895982F909580916B02892395
:1018100080936B02089510926B02089590916A0272
:10182000982B90936A020895982F909580916A0260
:10183000892380936A02089510926A020895089598
:101840000E941F0C089590916002292F28232223C3
:1018500031F080958923809360020E94200C0895C6
:1018600008950E94300C089590916102292F282339
:10187000281729F0982B909361020E94310C08954B
:1018800090916102292F2823222331F0809589230A
:10189000809361020E94310C089580916102882337
:1018A00029F01092610280E00E94310C08950F939C
:1018B0001F93CF93DF930091040110910501C09114
:1018C0006B0280916A02C82BD0916102DD2331F056
:1018D0000E94A52181110E944D0CCD2BF801C083DF
:1018E000C0910401D091050148E050E067E572E045
:1018F000CE010E94072D892B59F088E0FE01A7E553
:10190000B2E001900D928A95E1F7CE010E944E213E
:10191000DF91CF911F910F9108950E94570C089568
:1019200008950E94900C089590911F0392FF11C09A
:1019300098E0899F90011124622B60935F020E94BE
:10194000160880915F028695869586950E94910C77
:1019500008950E941608089510925F0280E00E9488
:10196000910C089590915F028095892380935F0286
:10197000282F277021110DC0891759F090911F034E
:1019800092FF07C08695869586950E9426080E943C
:10199000AC0C089590911F0392FB222720F9281781
:1019A00069F080FB92F990931F0380911E03909140
:1019B0001F030E94120D82E00E94B20C08958091D4
:1019C0001F0382FB882780F991E089270E94CA0CB7
:1019D000089581E00E94CA0C089580E00E94CA0C1C
:1019E00008956FEF7FEF80E090E00E945F2D0895F3
:1019F00080E090E00E942B2D9C0181E0253E3E4F2F
:101A000009F080E0089582E090E00E941D2D089585
:101A100083E090E00E941D2D089584E090E00E94F4
:101A20002B2D0895BC0184E090E00E945F2D089565
:101A3000AB01BC018FE090E00E94532D0895AB01F3
:101A4000BC0183E190E00E94532D089560E070E0B6
:101A5000CB010E941F0D089560E070E0CB010E9451
:101A6000180D0E94260D0895A8E0B0E0EAE3FDE01D
:101A70000C94412C65EE7EEF80E090E00E945F2D9B
:101A800060E082E090E00E94412D81E090E0909340
:101A900015028093140261E083E090E00E94412DE2
:101AA00060E074E184E090E00E945F2D60E086E0F9
:101AB00090E00E94412D60E087E090E00E94412D7F
:101AC00040E050E0BA0188E090E00E94532D60E0D1
:101AD00083E290E00E94412D60E08CE090E00E9463
:101AE000412D60E08DE090E00E94412D19821A8224
:101AF0001B821C821D821E821F82188648E050E0D5
:101B000067E170E0CE0101960E94312D40E050E087
:101B1000BA018FE190E00E94532D0E942C0D28966F
:101B2000E2E00C945D2C0E94340D0895682F8EE045
:101B300090E00E94412D0895A6E0B0E0E2EAFDE0C9
:101B40000C943F2C0E94B2228C0180916C029091E7
:101B50006D028017910779F019821A820E94B222D1
:101B6000BC0149815A8180E090E00E94F10310930A
:101B70006D0200936C022696E4E00C945B2C0E94AC
:101B8000E21060937A0270937B0280937C029093C0
:101B90007D0260937602709377028093780290932F
:101BA00079020895089508950E94D20D0895089528
:101BB0000E94D70D089581E0089580E291E10E948E
:101BC00097150E94D30D0E94D40D08950E94F5121E
:101BD0000895089508950E94E90D0E94EA0D089560
:101BE0000E94F80C811102C00E94930D0E94030D07
:101BF00080937E020E940D0D90931F0380931E031D
:101C00000E94080D90E00E94DA07809112029091E4
:101C100013020E94FB0708950E94A9220E94AC10A3
:101C20000E94F8120E9435120E94F00D0E94C50316
:101C30000E94611F0E94A61C0E9414130E94D80DCE
:101C40000895A6E0B0E0E7E2FEE00C94382C0E9494
:101C5000DB0D81110CC00E949C0D0E94F5120E94A8
:101C6000F51D0E94D8032696EBE00C94542C0E949C
:101C700059128EE6A82E82E0B82E750110E0F70109
:101C800001917F01812F0E942A111F5F183009F4F2
:101C900043C00817A1F380917E0281FD0E9430119C
:101CA0000E94E60DC82E00E099249394802F0E9494
:101CB0002A11182FF50191915F01891739F1D82E5A
:101CC000D926F12CEE24E3948E2D8D218823B1F0BA
:101CD000CC20A1F0F9820A830E94B2229C838B83DC
:101CE0009D8291E08E2D8123811101C090E0498178
:101CF0005A816B817C818D810E94F103F394EE0CFB
:101D0000F7E0FF12E1CFF501319710830F5F083044
:101D100069F60E94BF0DA1CF0813BDCF9CCF1F93C2
:101D2000CF93DF930E94B90FEC01811522E5920752
:101D300008F053C0811540E5940708F0DDC0803EEF
:101D40009105F8F48D3C910508F0AEC0883A9105F4
:101D500080F4853A910508F099C08130910521F011
:101D60000497813A910550F4CE01DF91CF911F91F4
:101D70000895885A91094B9708F48BC0C0E0D0E0D1
:101D8000F3CF811550E49507F8F4C11580E2D80728
:101D900008F0CBC0C83ED10538F3CE019A95811525
:101DA0009F4160F78D2F0E945D10182FCE0199275B
:101DB0000E94B90F212F30E0322F2227E901CC27D2
:101DC000DF71C82BD92BD0CF99270E94B90FCC2710
:101DD000DF70C82BD92BD06AC7CF803842E5940773
:101DE000C8F5803652E5950708F067C0C03482E533
:101DF000D807B0F08C2F86958695877020E2829F59
:101E0000C0011124C37021E030E0A90102C0440FD9
:101E1000551FCA95E2F7EA01C82BD92BDC68A4CF7D
:101E2000C03252E5D50708F041C08C2F86958695C3
:101E300020E2829FC0011124C37021E030E0A9019B
:101E400002C0440F551FCA95E2F7EA01C82BD92BEF
:101E5000DD688ACF803C52E5950760F48F71C03A07
:101E6000D24508F03FC090E0982F8827EC01C46F5E
:101E7000D06A7ACF805C9245809708F07FCFDC2FC4
:101E8000CC27CC27DF71C06FD06A6ECFA497D06407
:101E90006BCFC85AD0E0CC0FDD1FC558DE4F09907C
:101EA000D881C02DD46460CFD0655ECFCF71D0E033
:101EB000DC2FCC27C16FD06A57CF86958695877067
:101EC00020E2829FC0011124C37021E030E0A9010B
:101ED00002C0440F551FCA95E2F7EA01C82BD92B5F
:101EE000DA6842CF0E945D10C82FD0E0DC2FCC27EB
:101EF000CC27DF71D06238CF8F710E945D1065E012
:101F0000D695C7956A95E1F7CF70D0E0DC2FCC2746
:101F1000282F30E084FF05C054E0220F331F5A956C
:101F2000E1F7C22BD32BD0691FCF8D2F8F710E9469
:101F30005D10182FCE0199270E94B90F212F30E094
:101F4000322F222722273F71282B392BE901D2CFAC
:101F5000462F672F783028F4473018F40E94BB02D0
:101F6000089580E090E008950E94A80F0E948F0ECF
:101F70000895803E9105D1F1C8F48133910509F4AB
:101F80007FC048F48932910509F46FC08A32910507
:101F900009F47DC0089589339105E1F082389105F7
:101FA000C9F08533910509F45BC00895843E91051D
:101FB000D1F148F4823E910531F1833E910541F122
:101FC00081EE90E00895863E9105C1F1873E91052E
:101FD000E1F1089520911E032370211165C0209125
:101FE0001F0323FF14C089E290E0089520911E038F
:101FF00020FD43C030911F0330FF09C024FF4EC0B5
:1020000080E090E0089520911E0322FDF7CF08950F
:1020100020911E0322FD45C030911F0330FD44C0B6
:1020200024FFF5CFEDCF20911F0321FFF0CF80914A
:102030001E0384FDE5CF87EE90E0089520911E03F6
:1020400023FFE5CF24FDDCCFF6CF20911E0323FD37
:102050002EC030911F0331FFE3CF84EE90E008954E
:1020600020911E0325FFD3CFBECF20911E0325FD57
:1020700021C020911F0323FFCACF89E390E0089578
:1020800020911E0326FFC3CF8AE290E0089520919D
:102090001E0326FFBCCF81E390E0089583EE90E01D
:1020A000089582EE90E0089580EE90E0089586EE27
:1020B00090E0089585E390E0AACF90911E0392FFEF
:1020C00010C041E0282F2471243009F040E031E0B5
:1020D000282F2871283009F030E0431711F02CE048
:1020E000822793FF10C041E0282F2471243109F08A
:1020F00040E031E0282F2871283109F030E0431703
:1021000011F02CE0822730911F0330FF10C051E006
:10211000282F2171213009F050E041E0282F28714B
:10212000283009F040E0541711F029E0822731FFF0
:1021300010C041E0282F2171213109F040E031E049
:10214000282F2871283109F030E0431711F029E0D9
:10215000822794FD877E0895109220031092210318
:1021600010922203109223030895CF92DF92EF92F0
:10217000FF92CF93DF9300D000D0CDB7DEB76B01D5
:102180007C010E94F512811112C00E94BE22698357
:102190007A838B839C83C61AD70AE80AF90AC0920D
:1021A0002003D0922103E0922203F09223030F90A8
:1021B0000F900F900F90DF91CF91FF90EF90DF90F5
:1021C000CF900895A4E0B0E0E8EEF0E10C94412C4B
:1021D0000E94F512882371F00E94BE2269837A83DF
:1021E0008B839C8369817A818B819C812496E2E038
:1021F0000C945D2C0E94BE2269837A838B839C831E
:102200008091200390912103A0912203B091230398
:1022100029813A814B815C81280F391F4A1F5B1F3E
:1022200029833A834B835C83DDCF0E94F512882398
:1022300019F00E94B22208950E94E210CB01089585
:1022400080E0089508950E942211089508950E9443
:1022500026110895E82FF0E0E35DFC4F808108959A
:10226000089580EA8A95F1F7089500C008950E94C4
:102270003111089508950E943A110895EF92FF9246
:102280001F93CF93DF9300D000D0CDB7DEB70E946D
:10229000F512182F60913503882309F447C01A827C
:1022A00019821C821B82862F90E09E012F5F3F4F78
:1022B0007901B901835D9C4F0E9422138823E9F0C4
:1022C0008091240390E044E050E0B701835D9C4F8F
:1022D0000E94072D21E020937F02892BC9F410E092
:1022E0000E942711812F0F900F900F900F90DF9178
:1022F000CF911F91FF90EF90089580917F028823E6
:1023000071F384E0F70111928A95E9F710927F0248
:10231000E0912403F0E0E35DFC4F89819A81AB8179
:10232000BC8180839183A283B383DACF70E0635D45
:102330007C4F8091240390E0835D9C4F0E94AB13FF
:102340000E943B11CFCFF894E82FE295EF70F0E0B8
:1023500041A18F7021E030E0B90102C0660F771F04
:102360008A95E2F7CB01962F9095942391A392A1A1
:10237000892B82A378940895CF93DF9384EF0E94F2
:10238000A31187E90E94A31186EC0E94A31184E3A4
:102390000E94A311C1EBD1E089918F3F11F00E94FF
:1023A000A31181E0C83BD807B9F7DF91CF91089519
:1023B000A0E0B0E0EEEDF1E10C943B2CEC01D62E68
:1023C000062F10E0C80188549E4F7C01FC018081DB
:1023D0008F3F09F445C0F894E82FE295EF70F0E0E4
:1023E00091A18F7021E030E001C0220F8A95EAF7B9
:1023F000892F822B81A382A12095282322A3789460
:102400000E943511E1EBF1E091E0C12C81918F3F09
:1024100081F0A82FA295AF70A05EB0E02C9130E0C3
:102420008F7002C0359527958A95E2F72170892F24
:10243000211180E0C82A990F81E0E83BF80731F7C5
:10244000F70180818F3F11F00E94A31161E0C1105C
:1024500001C060E08D2D0E943711C00FD11FC882CE
:10246000CDB7DEB7E8E00C94572C8091060180913F
:10247000060191E08927880F880F8093350394E047
:10248000981B909324030E94BC1188E0EDE2F3E0D6
:10249000DF01982F1D929A95E9F7E5E2F3E0DF015D
:1024A0001D928A95E9F784E00E949A120E942311F6
:1024B0000895A8E0B0E0EFE5F2E10C943E2C1A821A
:1024C0001982FE01339686E0DF011D928A95E9F7B5
:1024D000F12C8E010F5F1F4F6F2DC8010E94D81184
:1024E000F394B4E0FB12F8CF48E050E0B80185E285
:1024F00093E00E94072D21E0892B99F420E0609160
:10250000350370E0635D7C4F44E085E293E00E9418
:102510009B12182F0E943E11812B2896E5E00C9407
:102520005A2C88E0F801A5E2B3E001900D928A955B
:10253000E1F7E5CF0895A0E0B0E0E1EAF2E10C9424
:102540003B2CD82EE92EF62ED72F042FC22F222374
:1025500079F081E0809382020E94B22290938102FE
:102560008093800280E0CDB7DEB7E8E00C94572C72
:10257000C0908202CC20B1F38091800290918102C0
:102580000E94DB22059770F310E0A8016D2D7E2DCF
:102590008F2D9D2F0E94072D892B41F0A8016D2DB5
:1025A0007E2D8F2D9D2F0E94142DCC2D10928202F6
:1025B0008C2FD9CF52985A988FE891E00197F1F774
:1025C00000C0000089B182FB882780F90895CF936D
:1025D0000E94892BC82F811102C00E94842B8C2F4E
:1025E000CF91089580918602089580918502089583
:1025F0000E94E712809385020E94DA12809386027D
:102600000E94F212809306010E94F21267E0882372
:1026100049F080E00E9436160E94F51281110E9456
:102620005813089587E0F6CF0E94F512811102C079
:102630000E945B13089581E0909187029A3008F020
:1026400080E008950F931F93CF93DF93EC01162F33
:10265000072F809187028A3090F4612F702FCE016E
:102660000E94A813811121C0809187028F3FB1F48D
:102670000E94B222909384028093830209C08091C9
:102680008302909184020E94DB22843F914028F7CC
:1026900080E0DF91CF911F910F9108958F5F80931C
:1026A00087028A3028F781E0F4CF10928702FBCFAF
:1026B0000E94A42308950E94A7230895A0E0B0E0FB
:1026C000E4E6F3E10C943B2CFA0169017801C82F90
:1026D000880FDD0B3097B1F0DE0193E0AA0FBB1F2E
:1026E0009A95E1F7A95FBE4F11968D919C91129733
:1026F00088579D4F4C9150E0E417F50708F4AF015F
:102700000E94142DCE010E949224182F8823D1F00C
:10271000E114F104B9F083E0CC0FDD1F8A95E1F7F5
:10272000FE01E95FFE4F438150E0E416F50608F430
:10273000A701C95FDE4F6C817D8168577D4FC6015F
:102740000E94142D812FCDB7DEB7E8E00C94572CF2
:102750000E94101508950E9434150895A8E0B0E075
:10276000E4EBF3E10C943F2C8091A8029091A90234
:10277000A091AA02B091AB02BC01CD010E94EA2255
:1027800011E0643671058105910520F10E94E21087
:10279000DC01CB010296A11DB11D89839A83AB8315
:1027A000BC8300E010E020E030E044E050E0BE01F7
:1027B0006F5F7F4F82E00E945E13182F882351F0D5
:1027C0000E94BE226093A8027093A9028093AA027D
:1027D0009093AB02812F2896E4E00C945B2CAFE041
:1027E000B0E0E5EFF3E10C943E2C8E010F5F1F4F3C
:1027F000C8010E94BD1BFB848091AC029091AD0288
:10280000A091AE02B091AF02BC01CD010E94EA22BC
:102810006C877D878E879F87B8018C859D85AE8567
:10282000BF8584369105A105B10510F4FF20A9F0FC
:1028300000E010E020E030E04BE050E083E00E9458
:102840005E13882369F00E94BE226093AC027093ED
:10285000AD028093AE029093AF020E94BA1B81E05A
:102860002F96E5E00C945A2C8F929F92AF92BF92D4
:10287000CF92DF92FF920F931F93CF93DF93CDB749
:10288000DEB729970FB6F894DEBF0FBECDBF6B0140
:10289000A090BC01B090BD0101E010E09E012B5F53
:1028A0003F4F40E050E060E070E080E00E945E1347
:1028B000F82E882309F459C045018FEF881A980A29
:1028C0008091A4029091A502A091A602B091A702C6
:1028D000BC01CD010E94EA226E837F83888799879D
:1028E000643671058105910570F104E010E09E01E8
:1028F0002F5F3F4F40E050E060E070E081E00E94D9
:102900005E13182F64E070E0C4010E94621F9D8175
:1029100098132BC0112349F10E94BE226093A40298
:102920007093A5028093A6029093A70289819A8151
:10293000AB81BC818093A0029093A102A093A202DC
:10294000B093A30213C064E070E0C4010E94621F50
:102950009D818913CACFF50181819281A381B481C0
:1029600089839A83AB83BC83E1CFF12C8091A00251
:102970009091A102A091A202B091A302F6018083DE
:102980009183A283B3838F2D29960FB6F894DEBF6F
:102990000FBECDBFDF91CF911F910F91FF90DF90C0
:1029A000CF90BF90AF909F908F900895A0E0B0E03F
:1029B000ECEDF4E10C94392CF82EE92EB62EA72E6E
:1029C0008A010E941B13CC24C394D12C882319F0B4
:1029D0008AE0C82ED12CC1E0D0E06B2D7A2D8F2D4E
:1029E0009E2DF8010995811116C02196CC16DD06A1
:1029F00094F0CC9FC001CD9F900D900D112420E04C
:102A000030E045E34A95F1F700002F5F3F4F28176C
:102A10003907B9F7E2CFCDB7DEB7EAE00C94552C11
:102A20000F931F93CF93DF93D82FC92F8B0144E3CC
:102A300054E10E94D614811106C080E0DF91CF914D
:102A40001F910F9108954EEA53E1B8018D2F9C2FED
:102A50000E94D614882389F34FEE53E1B8018D2FDD
:102A60009C2F0E94D614EACFABE0B0E0EAE3F5E198
:102A70000C943B2CFB010091BC011091BD01C801DD
:102A8000019624E0DC0101900D922A95E1F764E0C3
:102A900070E00E94621FF8018083658176818781E2
:102AA0009085C0909C02D0909D02E0909E02F09094
:102AB0009F026C157D058E059F0551F060939C0269
:102AC00070939D0280939E0290939F020E94B51086
:102AD0008BE0F8013996DE01119601900D928A95EE
:102AE000E1F7F801138A8B85882329F060E0CE0195
:102AF00001960E94EC1C2B96E8E00C94572C0E9447
:102B0000210E08950E944B220E9444260E94DD0D52
:102B10000E945E260E940C0E0E946B260E94702668
:102B20000E947F150E948A260E94EB0DF7CF90939A
:102B3000EF018093EE010895A0E0B0E0E2EAF5E154
:102B40000C94392CE82F71110DC0442321F0F0E0D2
:102B5000EA5EFC4F8491682F782FCDB7DEB7EAE0AC
:102B60000C94552C262F30E0C72FD0E0F0E0442302
:102B700021F0EA5EFC4FE491F0E086E0829F700174
:102B8000839FF00C11240FEF10E0C701B8010E94E1
:102B9000B02BAB01220F331F65E5649FC001659F19
:102BA000900D1124281B390BC22ECC0CC20EC8016B
:102BB0008C1B9D0B8E9F90018F9F300D9E9F300D23
:102BC0001124832FCC9EB001CD9E700D1124672F50
:102BD00077275801A61AB70AAE9ED001AF9EB00D56
:102BE000BE9EB00D11247B2F5801AC18B1086501B1
:102BF000CC9E5001CD9EB00CDC9EB00C1124AB2CB1
:102C0000BB240A191B090E9FE0010F9FD00D1E9FC8
:102C1000D00D11246E2F43305105C9F09CEFE916F9
:102C200093E0F90650F44130510509F496CF423053
:102C3000510589F07E2F6D2F90CF4430510571F0F2
:102C400046305105B9F3632F8B2F7E2F86CF6B2F24
:102C5000732F8E2F82CF732F8D2F7FCF7D2F632FDA
:102C6000F8CF41E00E949C1508950895EAE2F1E052
:102C70008083618308950E9431160895CF93DF9376
:102C8000982F762F842FE901692F0E943B167983B4
:102C900068838A83DF91CF910895809136038430D1
:102CA00028F4837084608093360308958C3AE8F3A7
:102CB0008370886AF8CF4F925F926F927F928F9263
:102CC0009F92AF92BF92CF92DF92EF92FF920F93BB
:102CD00088E090E00E94252D2B013C0183E290E0EA
:102CE0000E941D2D282F30E040E050E060E070E0B1
:102CF00080E090E000E20E94682C53014201C12C68
:102D0000D12C7601242939294A295B296C297D296E
:102D10008E299F290F91FF90EF90DF90CF90BF9069
:102D2000AF909F908F907F906F905F904F9008959D
:102D3000A0E0B0E0EEE9F6E10C943B2C8901D42F41
:102D4000C52F6B017C010E944D16A8016D2F7C2FB1
:102D500088E090E00E94532D98014D2F5C2FB60122
:102D6000C70100E20E94832C622F83E290E00E9460
:102D7000412DCDB7DEB7E8E00C94572CE6E3F3E045
:102D800085E0808311828FEF828383831482A3E0A6
:102D9000B3E012968C911297836012968C93758192
:102DA00025E030E04FEF5FEF60E0868197810E9481
:102DB000981608958091360380FF03C08695869506
:102DC000089580E0089590913A03933018F49F5F3E
:102DD00090933A03882391F0209136033091370382
:102DE000409138035091390360913A0370913B034D
:102DF00080913C0390913D030E949816089581E0D4
:102E00000E94E316089590913A03992319F0915086
:102E100090933A03882391F0209136033091370341
:102E2000409138035091390360913A0370913B030C
:102E300080913C0390913D030E949816089581E093
:102E40000E940317089560912B018091360380FF43
:102E500011C070E020912A0130E0C901880F991F4C
:102E6000820F931FE091EB01F091EC01825C9C4F8B
:102E70000995089580912C0190912D01282F30E023
:102E8000F901EE0FFF1FE20FF31FE25CFC4F891701
:102E900000F71182108212828F5F3396F8CF9091E3
:102EA000360390FF11C090912C0150912D01292FD4
:102EB00030E0F901EE0FFF1FE20FF31FE25CFC4F61
:102EC000951718F00E942317089581836083428329
:102ED0009F5F3396F5CFA3E0B0E0E1E7F7E10C9414
:102EE000412C9091360390FF0AC09E012F5F3F4F07
:102EF0000E943E164B8169818A810E944F1723965A
:102F0000E2E00C945D2CCF93DF93EC01EC81F0E0D8
:102F1000EF5EFD4F4491E6E3F3E0628181810E9420
:102F20006B178C818F5F8C83DF91CF910895CF9346
:102F3000DF93EC01E6E3F3E0438162818C810E9440
:102F40006B178C818F5F8C83DF91CF910895A3E005
:102F5000B0E0EDEAF7E10C943F2C8C018091B002D7
:102F600081110AC09E012F5F3F4F4FEF6FEF0E940C
:102F70003E168A818093B002F8016481613049F085
:102F80006230D1F08091B00240E0662331F040E041
:102F900015C06091B00240E080E00E944F17F80138
:102FA000848190E0019663E070E00E94C42B8483EA
:102FB0002396E4E00C945B2C4091B00280E060E04A
:102FC000ECCFA3E0B0E0E7EEF7E10C94392CE82E6B
:102FD000D62EF42EB22E9091360390FF42C030913F
:102FE0003703381308C080913803861304C08091DA
:102FF0003903841729F080910503826080930503CB
:10300000E92FE695E695AE2FB0E0A254BE4F8C9125
:10301000809303039C7F943041F59E012F5F3F4FC7
:103020004F2D6D2D8E2D0E943E164B8169818A8118
:103030000E944F173E2D30933703D0923803F09201
:103040003903BB2071F02091360360913A037091EF
:103050003B034D2D5F2D80913C0390913D030E94D9
:1030600098162396EAE00C94552C823019F4F090CF
:103070003903E0CF8630F9F28930E9F28931D1F6AF
:10308000E9518E2F8170A82EE695F0E0EF5EFC4F9F
:10309000E491C12C0E2F10E060912E01C61618F09D
:1030A0000E942317C7CF2C2D30E0C09EC001C19EC7
:1030B000900D112470E00E94B02B8E2DA11013C032
:1030C000860F90912C01A901490F511D9A01220FE1
:1030D000331F240F351F225C3C4F4F2D6D2D0E9456
:1030E0003E16C394D9CF861BECCF282FE6E3F3E03E
:1030F000818143816281885F0E94E117089581E0A8
:103100000E9475180895282FE6E3F3E0818143813A
:10311000628188500E94E117089581E00E9483181F
:103120000895282FE6E3F3E0628131E1630F08F4AC
:103130006FEF438181810E94E117089581E00E9431
:1031400091180895282FE6E3F3E0628131E1631BD3
:1031500008F460E0438181810E94E117089581E0D5
:103160000E94A2180895282FE6E3F3E0438131E19D
:10317000430F08F44FEF628181810E94E1170895A7
:1031800081E00E94B3180895282FE6E3F3E043811D
:1031900031E1431B08F440E0628181810E94E11724
:1031A000089581E00E94C418089520E00E94E1176C
:1031B0000895EF92FF921F93CF93DF93EC0110E0FD
:1031C000EE24EA94F12C60912E01161770F00E9403
:1031D00023179A818C8190FF25C08F5F8C83DF91AC
:1031E000CF911F91FF90EF90089580912C01810F56
:1031F0009927991F9C01220F331F280F391F225C2A
:103200003C4F70E0C7010E94C42B962F8C814091E7
:10321000390360913803199F800D11240E943E16D6
:103220001F5FD1CF8150DACFA0E0B0E0EAE1F9E151
:103230000C94382CEC018C819A8190FD0EC0BB243B
:10324000B39481110EC080912E018150BB24B394A0
:103250008093B20281E08C8304C0BB24BA9488239B
:10326000B9F3A12C80912E01A816B8F00E94231763
:103270009091B20281E0B81256C080912E01815027
:10328000992319F08FEF890F91E08093B2029C830C
:10329000CDB7DEB7EBE00C94542C80912C01CA2CF6
:1032A000D12C8C0D9D2D911D8C01000F111F080F2D
:1032B000191F025C1C4FF80111821082128234E047
:1032C000E32EF12C912C8091B202890D8F302CF1DC
:1032D0006EE00E94A22B892F082E000C990BC816B5
:1032E000D90691F4809139038E9DA0018F9D500DD8
:1032F0001124559547955595479598016091380348
:10330000809137030E943E169B0CF1E0EF1AF10802
:10331000E114F104C1F6A394A5CF87FFDDCF90910E
:103320002E01890FD9CF892F90E0019660912E014F
:1033300070E00E94C42B982FA8CF1F93CF93DF93E8
:10334000EC018C81811109C081E08C831092B10263
:1033500092E0909329018093280180912C01909113
:103360002D01282F30E0F901EE0FFF1FE20FF31FB0
:10337000E25CFC4F891748F110E060912E011617AE
:1033800050F10E942317809128012091B102280F4B
:103390002093B10290912901980F90932901191659
:1033A00054F4022E000C330B40912E014150550B6A
:1033B0002417350734F0819580932801813009F472
:1033C0001C82DF91CF911F91089511821082128289
:1033D0008F5F3396CFCF212F30E070E0C9010E947C
:1033E000C42B90912C01980F892F90E04091B1024D
:1033F000042E000C550BFC01EE0FFF1FE80FF91F08
:1034000024173507ACF040912901042E000C550B10
:10341000421753076CF09F01225C3C4F40913903E7
:1034200060913803809137030E943E161F5FA5CF3D
:10343000E25CFC4F118210821282F8CFAEE0B0E065
:10344000E4E2FAE10C943D2C8D879E87AD85BE8524
:1034500014961C91212F30E0D9010E94082C9B0169
:10346000AC010E941E2C69837A838B839C83E0E2EB
:10347000F0E0E11BF109A5E5B0E09B01AC010E9481
:103480001E2C69877A878B879C879F01DF010E94AA
:10349000002C9B01AC010E94292C6D837E838F83BD
:1034A00098879B01AC0189819A81AB81BC81280FEF
:1034B000391F4A1F5B1F69857A858B859C850E9411
:1034C000D82B022F30E00A3248F5A901440F551FCE
:1034D000420F531F55954795142F1095F12C85E5F4
:1034E000E82EE01A80912E01F81630F10E94231781
:1034F000AD85BE8514969C9181E0992319F0903298
:1035000019F48FEF8093270180912701890FED85B2
:10351000FE8584832E96E6E00C94592C85E590E098
:10352000821B930BAC01440F551F480F591F57FFC7
:10353000D1CF4F5F5F4FCECF8E2DF1FC802F4091CA
:103540002C014F0D5527551F9A01220F331F240FB1
:10355000351F225C3C4F412F609138030E943E167C
:10356000F394C0CF0F931F93CF93DF93EC0100E050
:1035700010E040912E01842F90E0081719076CF09D
:103580000E9423178C8190E00196817099278C838B
:10359000DF91CF911F910F91089580912C01800FA1
:1035A000912F911D9C01220F331F280F391F225C80
:1035B0003C4F9C816091380380913703469550E0E1
:1035C000041715074CF4992349F0409139030E94E0
:1035D0003E160F5F1F4FCDCF9923B9F340E0F7CFD1
:1035E000A0E0B0E0E6EFFAE10C94332CFC0162803D
:1035F000448081E08483E1E1F2E07490E0E9F2E06C
:10360000E491C0913903C695C158D0E0CC0FDD1FBD
:10361000CD2FDD27812C75E0972EAA24AA94B12CFA
:1036200055245A94E719EE2EF12C80912E0188161C
:1036300038F00E942317CDB7DEB7E0E10C944F2C91
:10364000C82CD12C82E0861568F09C9CF0019D9CD2
:10365000F00D1124EA54FD4F80913703808380914F
:1036600038038183411023C09C9CF0019D9CF00D88
:103670001124EA54FD4F1382128280912C018C0D8B
:103680009D2D911D9C01220F331F280F391F225C95
:103690003C4F9C9CF0019D9CF00D1124EA54FD4F81
:1036A0004281618180810E943E168394BECF9C9CA2
:1036B00080019D9C100D11240A541D4FF801838137
:1036C0008823F1F081508383589EC00111246481C6
:1036D00070E00E94B02BFB01FF27EF5EFD4F84914D
:1036E000E82FE7195E9EC0011124B7010E94B02B9C
:1036F00080913903689FB0011124F8017283BDCF16
:103700000E94EA2CB5010E94C42B8C179D070CF077
:10371000B4CFF2E0F61598F40E94EA2CB5010E94AD
:10372000C42BF80180830E94EA2C2091380326954F
:10373000622F70E00E94C42B280FF80121839C9C0B
:10374000F0019D9CF00D1124EA54FD4F12828091EE
:103750003903893C58F088EC9C9CF0019D9CF00D4D
:103760001124EA54FD4F8483838387CF8431A0F7EB
:1037700084E1F2CF109205030895CF93DF93EC011B
:1037800088E0E6E3F3E0DE0101900D928A95E1F72F
:103790008091030390910403A09105038887998782
:1037A000AA87DF91CF910895E3E0F3E0118282814F
:1037B000846082830895E6E3F3E080818E7F8083D6
:1037C0000E94D41BE3E0F3E08281816082830E9447
:1037D00023170895E6E3F3E020812E7F20833181D3
:1037E0004281538164817581868197810E949816F8
:1037F0000E94D41BE3E0F3E08281816082830E9417
:1038000023170895609136036695669570E04BE046
:1038100050E08FE291E00E94FA2C892B19F481E0AC
:10382000809304030E9415119093FD028093FC0283
:103830008091050384608093050308959091360379
:1038400090FF3FC08823F1F18B32F0F58F73282F62
:10385000220F220F809136038370282B209336038A
:1038600080910503816080930503662381F0309188
:103870003703409138035091390360913A037091B6
:103880003B0380913C0390913D030E949816609108
:1038900036036695669570E04BE050E08FE291E06C
:1038A0000E94FA2C892B91F00E94D41B81E0809316
:1038B000FF024091390360913803809137030E94E1
:1038C000D518089581E0C3CF8AE2C1CF0E94021CBF
:1038D000EDCF682F80913603869586958F5F8B326A
:1038E00008F081E00E941E1C089581E00E94691C7E
:1038F0000895682F90913603969596958FEF890FCE
:10390000913009F48AE20E941E1C089581E00E9411
:10391000791C089561E00E941E1C0895E6E3F3E01F
:10392000808181608083869586950E948A1C089597
:103930008091360380FF03C00E94EA1B08950E9415
:103940008E1C089560E00E941E1C08958091020361
:10395000811141C00E945B162093360330933703D8
:10396000409338035093390360933A0370933B03B9
:1039700080933C0390933D03809105038360809383
:1039800005032430A0F40E94BE160E945B1620930B
:1039900036033093370340933803509339036093D1
:1039A0003A0370933B0380933C0390933D030E9442
:1039B0004D160E94D41BE091E901F091EA010995AE
:1039C0008091360380FF04C0869586950E94A21CD4
:1039D00081E08093020308951F93CF93DF93EC015E
:1039E000162F8A8580FF0DC0888180FF25C08091B9
:1039F00036038160809336038881869586950E9480
:103A00001E1C8A8581FF06C0212F4B816A81898116
:103A10000E94E1178A8582FF05C08985882379F095
:103A20000E94021C8A8583FF03C081E08093FF020D
:103A3000DF91CF911F9108950E94DB1BE2CF0E947E
:103A4000D41BF0CFEF92FF920F931F93CF93DF938E
:103A500080910403882309F465C080910303E091F9
:103A60003603E695E695E81BE093FE02823009F006
:103A70005EC0F0E0E35FFD4FE491CE2FD0E003E8BD
:103A800017E18091FF02882361F01092FF020E94EB
:103A900015119093FD028093FC0210920103109285
:103AA00000030E9415119C018091FC029091FD027F
:103AB000A901481B590B4F3F5F47A0F54091B50244
:103AC0004423B1F01092B5024091B3025091B40278
:103AD000241B350B2F3F3F4758F4405D5A48509305
:103AE000B4024093B302209105032860209305039C
:103AF000E0900003F09001038C0F9D1F9093FD0256
:103B00008093FC028CEF92E0F8010995809100030C
:103B100090910103892B31F4E114F10419F081E053
:103B20008093B502CDB7DEB7E6E00C94592CC8E21D
:103B3000D0E00EE11AE1883109F4A3CFC0F48F3050
:103B400009F43AC048F4863021F1893059F1C0EDCA
:103B5000D7E005E316E195CF8531C9F7F0E0EF5FD7
:103B6000FD4FE491CE2FD0E00DE919E18ACFC4EFEB
:103B7000D1E002EB1AE1843209F483CF853231F1CE
:103B8000833229F7EFEFF1E0C591D49107EA17E10D
:103B900078CFF0E0E65FFD4FE491CE2FD0E007E96B
:103BA00017E16FCFE695F0E0E95FFD4FE491CE2F8E
:103BB000D0E009ED18E165CFE695F0E0EC5FFD4F50
:103BC000E491CE2FD0E004E119E15BCF8E2F63E0CA
:103BD0000E94962BE92FF0E0E450FE4FE491CE2FA7
:103BE000D0E000EF1AE14DCF08950E94221D089504
:103BF000FA01882311F009950895FB01FCCFCF93BA
:103C0000DF93C82FD62F0E94DA168C1748F00E9437
:103C1000DA168D1728F40E94751CDF91CF91089554
:103C20008C2F0E948A1CF9CF1F93CF93DF93EC0156
:103C3000FB011581111168C00E94FA0B8272FE010E
:103C4000E052F847E531F10508F05EC0EA56F24D62
:103C50000C94FA2B0E94981C812FDF91CF911F9119
:103C6000089546E85CE165E77CE10E94F81DF4CF29
:103C700045E75CE166E87CE1F8CF4DE858E16FE7A5
:103C800078E1F3CF4FE758E16DE878E1EECF4FEA06
:103C900058E16EE978E1E9CF4EE958E16FEA78E161
:103CA000E4CF41ED58E160EC78E1DFCF40EC58E142
:103CB00061ED78E1DACF4FE157E16FEF76E1D5CFF3
:103CC0004FEF56E16FE177E1D0CF81E00E948A1C8F
:103CD000C3CF65E082E00E94FF1DBECF68E086E0B2
:103CE000FACF6EE089E0F7CF64E18FE0F4CF67E1CF
:103CF00085E1F1CF88E1EACF62E289E1ECCF83E2AE
:103D0000E5CF6AE285E2E7CF11E0A6CF539A0895A6
:103D10009C01AB016BB1677F7BB17860EFB7F89422
:103D2000CA01880F991F840F951F820F931F821756
:103D3000930741F4EFBF8FE594E00197F1F700C0DE
:103D400000000895D9014D919D0158E07BB9000014
:103D500000C047FF6BB9440F000000C000C000C0A6
:103D60006BB900C05A9591F7E2CF8B3258F4853089
:103D700090F0EBEFE80FE63270F4F0E0E555F24D2D
:103D80000C94FA2B833448F48A3308F051C08533FD
:103D900031F0883369F080E008958334E1F781E001
:103DA00090E00E94DA070E948B0702C00E94930DE8
:103DB00081E0089580917E02807F80937E0281E081
:103DC00080930603F5CF0E943B03F2CF90917E02D1
:103DD000892F8E7F90FF816080937E0280FDE8CFE7
:103DE000817F80937E02E4CF90917E02892F8D7F28
:103DF00091FF826080937E0281FFDACF80917E0204
:103E00008160EFCF90917E02892F8B7F92FF84603B
:103E100080937E0282FDF2CFCBCF90917E02892FDC
:103E2000877F93FF886080937E0283FDE7CFC0CFBA
:103E3000895321E030E0A90102C0440F551F8A9543
:103E4000E2F7CA01AECF8D51F4CF80E008950E9411
:103E5000251F0895CF93C82F80910603882331F042
:103E6000813099F01092060380E00DC00E94FA0B99
:103E70008232D1F78C2F0E94251F811118C08C2F00
